:10E00000B240805A20013F4002000F9305242F8325
:10E010009F4F98E50002FB233F4002000F9304242A
:10E020001F83CF430202FC233040FAE0304030E04F
:10E0300000130F12D2B32B00022492D30202B1C0FC
:10E04000D0000200C2432B003F4100130F12F2B276
:10E0500023000224A2D30202D2B323000224A2D2BC
:10E060000202B1C0D0000200C24323003F410013AE
:10E070000E430E9F132C0343034303430343034305
:10E080000343034303430343034303430343034360
:10E090000343034303431E530E9FED2B3041B24015
:10E0A000805A2001F24036002100F240060029008B
:10E0B000C2431900C2432600C2432E00C2431B00C4
:10E0C000F240D2FF2200F240FAFF2A00F2431A0087
:10E0D000F24009002400D2432C00F2400900250040
:10E0E000D2432D00F2D007005700F2D0E0FF5600D7
:10E0F000D24358003041475052003140B002B01274
:10E100009EE03E4050000F41CF4300001F531E834E
:10E11000FB23824302023F40FF00B01270E0F2E0B6
:10E12000100019003F40FF00B01270E0F2E0100054
:10E13000190082430202C2432B00C243230032D2A1
:10E140004A4392B302022C245A43D2B32800282017
:10E1500032C2F2D0200019000E415F43B01248E2F3
:10E160004B4FD2C32B00F2F0DFFF1900F2D01000AA
:10E1700019003D4003000E413F40F6E0B01266E555
:10E180000F9356204D4B0E417F400300B012AEE37B
:10E19000D2C32300F2F0EFFF190032D292C3020281
:10E1A000A2B302021E2432C25A43F2D01000190058
:10E1B0000E416F43B01248E2F2C22300F2F0EFFFCB
:10E1C0001900F2D0200019004D4F0E415F43B012EC
:10E1D000AEE3D2C32B00F2F0DFFF1900A2C30202AC
:10E1E00032D2A2B202021F2432C25A43F2D010002D
:10E1F00019000E417F400300B01248E2D2C3230051
:10E20000F2F0EFFF1900F2D0200019004D4F0E413F
:10E210005F43B012AEE3D2C32B00F2F0DFFF190070
:10E22000A2C2020232D24A938B2332D0D000883F5E
:10E230004D4B0E416F43B012AEE3F2C22300AA3F32
:10E2400031505000304096E50B120A1209120812A4
:10E2500007120612051204122182814E0000494362
:10E260000C430D438F112F9390243F900300813472
:10E270001F9303243F40FF00903C64435B4366428E
:10E2800045433E4028003A4029006F4E8F11474BCE
:10E290000FF70F975C24484478E3CAF80000B240B7
:10E2A000085A20017B424D46464549596F4E8F1111
:10E2B0000FFD0F9DFB276F4E8F110FF70C460C9330
:10E2C00003240F111C83FD2349DFCAD400006F4EC5
:10E2D0008F110FFDFC27CAF800007B53E623C149CC
:10E2E0000200C14303000543919302002824B24079
:10E2F000085A20017B4249596F4E8F110FFD0F9D27
:10E30000FB276F4E8F110FF70C460C9303240F1150
:10E310001C83FD2349DFCAD400006F4E8F110FFD0F
:10E32000FC27CAF800007B53E6232F410F55CF4945
:10E33000000015531F4102003F53059FD82BCAD43C
:10E340000000B240805A20011F410200263C1C53AD
:10E350000D633C9020A103203D90070006246F4EE2
:10E360008F110FF70F97F327963FB240085A2001FD
:10E37000F63F3F9003007E2364435B436642454380
:10E380003E4020003A402100803F744010007B4214
:10E390007640200075400300F33F2152344135415F
:10E3A00036413741384139413A413B4130410B1206
:10E3B0000A120912081207120612051204123180FD
:10E3C0000A00814E0000C14D0200084309438F112D
:10E3D0002F93B6243F900300A3341F9302243F439E
:10E3E000B73C64435C4365427E4006003D402800E4
:10E3F0003A402900B1402A0006006F4D8F117CF38E
:10E400000FFC02200F43A43C1F410600CFD50000A3
:10E41000474477E3CAF700006F4D8F110FFC0F9C44
:10E420006D245B410200B240085A20017942464EF9
:10E43000484578E36F4D8F110FFC0F9CFB274F4B26
:10E440007FF080FF7FF30E460E9303240F111E838F
:10E45000FD234FF4CADF0000CAF800006F4D8F1192
:10E460000FFCFC27CAD50000CAF700004B5B7953AC
:10E47000E123D14102000800C143090081430400A7
:10E48000919308002F24B240085A20012F411F51B8
:10E4900004006B4F79426F4D8F110FFC0F9CFB27CF
:10E4A0004F4B7FF080FF7FF30E460E9303240F1136
:10E4B0001E83FD234FF4CADF0000CAF800006F4D31
:10E4C0008F110FFCFC27CAD50000CAF700004B5B78
:10E4D0007953E123915304001F4108003F53819F6A
:10E4E0000400D12B1F410600CFF8000044D5CAD448
:10E4F0000000B240805A20011F432A3C1853096390
:10E50000389020A103203990070006246F4D8F1109
:10E510000FFC0F9CF327853FB240085A2001F63FBD
:10E520003F9003005C2364435C4365427E400600E9
:10E530003D4020003A402100B140220006005D3FEE
:10E54000744010007C42754020007E400300F03F84
:10E5500031500A0034413541364137413841394163
:10E560003A413B4130410B120B4D0D930A240C4FA5
:10E570000D4E6E4D1D536F4C1C534F9E04203B534C
:10E58000F8230C43053C5C4CFFFF5F4DFFFF0C8FF5
:08E590000F4C3B413041FF3FFD
:02E59800010080
:10FFE0002CE02CE04CE032E02CE02CE02CE02CE08B
:10FFF0002CE02CE02CE02CE02CE02CE02CE000E0CD
:040000030000E00019
:00000001FF
